:100000000C94C2000C94EA000C94EA000C94EA00F0
:100010000C94EA000C94EA000C94EA000C94AB0CEB
:100020000C94EA000C94EA000C94EA000C94C80EBC
:100030000C94EA000C94EA000C94EA000C94EA0098
:100040000C945F0D0C94EA000C942D0D0C94070D8C
:100050000C94EA000C94EA000C94EA000C94EA0078
:100060000C94A90D0C94EA0007634236B79BD8A7FD
:100070001A39685618AEBAAB558C1D3CB7CC5763CD
:10008000BD6DEDFD753EF6177231BF000000803F7B
:1000900008000000BE922449123EABAAAA2ABECD97
:1000A000CCCC4C3E00000080BEABAAAAAA3E000009
:1000B0000000BF000000803F000000000008417801
:1000C000D3BB4387D1133D190E3CC3BD4282AD2B38
:1000D0003E68EC8276BED98FE1A93E4C80EFFFBE30
:1000E00001C4FF7F3F00000000004E414E494E49D1
:1000F0005459494E46CDCCCC3D0AD7233C17B7D1F5
:100100003877CC2B329595E6241FB14F0A0000209A
:10011000410000C84200401C4620BCBE4CCA1B0E19
:100120005AAEC59D7400000000240027002A00007C
:10013000000000250028002B00020000000800023B
:1001400001000003040700000000000000000000A0
:10015000000023002600290004040404040404040D
:100160000202020202020303030303030102040862
:100170001020408001020408102001020408102011
:10018000C90F7E1911241FBECFEFD8E0DEBFCDBF4F
:1001900011E0A0E0B1E0ECE5F3E402C005900D92BF
:1001A000AC35B107D9F724E0ACE5B1E001C01D9250
:1001B000A736B207E1F710E0C1ECD0E004C0219708
:1001C000FE010E94A91FC03CD107C9F70E94DD10A3
:1001D0000C94A1210C9400008091980290919902B6
:1001E000891B990B089508950895AF92BF92CF92FD
:1001F000DF92EF92FF920F931F93CF93DF936C01E7
:100200007B018B01040F151FEB015E01AE18BF08C7
:10021000C017D10759F06991D601ED91FC91019079
:10022000F081E02DC6010995892B79F7C501DF9191
:10023000CF911F910F91FF90EF90DF90CF90BF90E3
:10024000AF900895FC01538D448D252F30E0842F0D
:1002500090E0821B930B541710F0CF9608950197EE
:100260000895FC01918D828D981761F0A28DAE0FDB
:10027000BF2FB11D5D968C91928D9F5F9F73928F62
:1002800090E008958FEF9FEF0895FC01918D828D8E
:10029000981731F0828DE80FF11D858D90E008955B
:1002A0008FEF9FEF0895FC01918D228D892F90E0B3
:1002B000805C9F4F821B91098F73992708958AE074
:1002C00093E00E94530121E0892B09F420E0822F62
:1002D000089580E090E0892B29F00E945F01811150
:1002E0000C9400000895FC01A48DA80FB92FB11D36
:1002F000A35ABF4F2C91848D90E001968F7399275C
:10030000848FA689B7892C93A089B1898C91837039
:1003100080648C93938D848D981306C00288F38932
:10032000E02D80818F7D80830895EF92FF920F935F
:100330001F93CF93DF93EC0181E0888F9B8D8C8D91
:1003400098131AC0E889F989808185FF15C09FB785
:10035000F894EE89FF896083E889F9898081837048
:10036000806480839FBF81E090E0DF91CF911F91F7
:100370000F91FF90EF900895F62E0B8D10E00F5F18
:100380001F4F0F731127E02E8C8D8E110CC00FB6EE
:1003900007FCFACFE889F989808185FFF5CFCE0186
:1003A0000E947301F1CFEB8DEC0FFD2FF11DE35A8D
:1003B000FF4FF0829FB7F8940B8FEA89FB89808109
:1003C0008062CFCF682F8AE093E00C949501CF93A1
:1003D000DF93EC01888D8823B9F0AA89BB89E8896D
:1003E000F9898C9185FD03C0808186FD0DC00FB613
:1003F00007FCF7CF8C9185FFF2CF808185FFEDCF91
:10040000CE010E947301E9CFDF91CF91089583302F
:1004100081F028F4813099F08230A9F00895873076
:10042000A9F08830C9F08430B1F4809180008F7DCC
:1004300003C0809180008F7780938000089584B5F9
:100440008F7784BD089584B58F7DFBCF8091B000F8
:100450008F778093B00008958091B0008F7DF9CFA1
:100460001F93CF93DF93282F30E0F901E65CFE4F16
:100470008491F901E459FE4FD491F901E85AFE4FF5
:10048000C491CC23A9F0162F81110E940702EC2FF2
:10049000F0E0EE0FFF1FE15DFE4FA591B4918FB725
:1004A000F894EC91111108C0D095DE23DC938FBF36
:1004B000DF91CF911F910895DE2BF8CF909100012D
:1004C00089130BC0E9E3F1E0E4919FEF9093000101
:1004D000E13049F028F0E23061F060E00C94300245
:1004E00010926E00FACF90916F009D7F90936F00F5
:1004F000F4CF909170009D7F9093700091E0909365
:10050000B0009091B100987F94609093B1001092E8
:10051000B300E3CFCF93DF9390E0FC01E459FE4FAB
:100520002491885A9E4FFC0184918823C9F090E061
:10053000880F991FFC01EB5DFE4FA591B491FC0162
:10054000E15DFE4FC591D49161110DC09FB7F89444
:100550008C91209582238C938881282328839FBFA8
:10056000DF91CF910895623051F49FB7F8943C9198
:10057000822F809583238C93E8812E2BEFCF8FB72A
:10058000F894EC912E2B2C938FBFEACF4F925F9271
:100590006F927F928F929F92AF92BF92CF92DF9293
:1005A000EF92FF920F931F93CF93DF9300D000D071
:1005B0001F92CDB7DEB78B0129013A01909100015E
:1005C0008917C9F09F3F09F47EC00F900F900F90DC
:1005D0000F900F90DF91CF911F910F91FF90EF90AF
:1005E000DF90CF90BF90AF909F908F907F906F9053
:1005F0005F904F900895E9E3F1E094919D8397FD1A
:10060000E4CF61E00E948A028D81882321F09D81E0
:10061000923009F04AC14801B12CA12C60E072E18E
:100620008AE790E0A50198010E945F1C29833A8324
:100630004B835C8369017A0181E0C81AD108E10823
:10064000F1089FEFC916D104E104F10409F00CF49C
:1006500001C160E472E48FE090E0A50198010E947E
:100660005F1C69017A0181E0C81AD108E108F1082C
:100670009D81923009F0A2C08FEFC816D104E10429
:10068000F10409F00CF4E6C160E970ED83E090E05C
:10069000A50198010E945F1C69017A0191E0C91AC5
:1006A000D108E108F1088FEFC816D104E104F10484
:1006B00011F00CF07FC183E09091B100987F892BFD
:1006C0008093B100CFC080930001E9E3F1E0949101
:1006D0009D839F3F09F479CF913041F150F09230E2
:1006E00009F446C09D8197FD70CF61E00E948A02A7
:1006F0008ECF14BC15BC94B5926094BD95B5916035
:1007000095BD282F30E0F901E85AFE4FE491F0E062
:10071000EE0FFF1FE15DFE4F45915491F901E45941
:10072000FE4FE491E093A8011D826BCF10928000F0
:100730001092810090918100986090938100909137
:100740008100916090938100282F30E0F901E85AF0
:10075000FE4FE491F0E0EE0FFF1FE15DFE4F45918B
:100760005491F901E459FE4FE491E093A70149CF78
:100770001092B0001092B1009091B00092609093EE
:10078000B0009091B10091609093B100282F30E0BB
:10079000F901E85AFE4FE491F0E0EE0FFF1FE15D32
:1007A000FE4F459154915093B2014093B101F9012C
:1007B000E459FE4FE491E093B30123CF9FEFC916B4
:1007C000D104E104F10409F00CF46DC068E478EEA2
:1007D00081E090E0A50198010E945F1C69017A0107
:1007E00081E0C81AD108E108F1089D81992309F434
:1007F000FAC08FEFC816D104E104F10411F00CF037
:10080000FBC0EFC064E274EF80E090E0A5019401CA
:100810000E945F1C69017A0181E0C81AD108E108D1
:10082000F10885E09FEFC916D104E104F10409F055
:1008300008F442CF62E17AE780E090E0A5019401FC
:100840000E945F1C69017A0181E0C81AD108E108A1
:10085000F108E5C081E09D8191112ECF95B5987F7B
:10086000892B85BD2FEF3FEFA9014114510461048D
:10087000710409F043C09D81913009F45EC092304B
:1008800009F46DC09111A1CEC7BC2093AD01309386
:10089000AE014093AF015093B00180916E00826031
:1008A00080936E0092CE82E0D6CFB12CA12C60E076
:1008B00072E18AE790E0A50198010E945F1C69013E
:1008C0007A0181E0C81AD108E108F108C114D10405
:1008D00091E0E906F10404F591E08D81813011F693
:1008E00080918100887F892B809381002FEF3FEFDB
:1008F000A9014114510461047104F9F0D801AA0F4F
:10090000BB1FA30192010E947E1C28EE33E040E051
:1009100050E00E94C81CAFCF68E478EE81E090E020
:10092000A50198010E945F1C69017A0181E0C81A43
:10093000D108E108F10893E0D0CFD0928900C092AD
:1009400088002093A9013093AA014093AB015093F2
:10095000AC0180916F00826080936F0036CEC092B0
:10096000B3002093B4013093B5014093B601509386
:10097000B7018091700082608093700026CE84E081
:100980009FEFC916D104E104F10409F008F466CF21
:10099000C980DA80EB80FC808AE0F594E794D794F4
:1009A000C7948A95D1F781E0C81AD108E108F10807
:1009B00085E054CF68E478EE81E090E0A5019801ED
:1009C0000E945F1C69017A0181E0C81AD108E10820
:1009D000F1089FEFC916D104E104F10411F00CF005
:1009E00011CF84E069CE83E09FEFC916D104E10402
:1009F000F10409F00CF432CF62E17AE780E090E094
:100A0000A50194010E945F1C69017A0181E0C81A66
:100A1000D108E108F1089D81992309F4B0CF86E05F
:100A20009FEFC916D104E104F10409F008F444CEA3
:100A3000C980DA80EB80FC809AE0F594E794D79443
:100A4000C7949A95D1F781E0C81AD108E108F10856
:100A500087E032CE82E030CE3FB7F8948091A30198
:100A60009091A401A091A501B091A60126B5A89BE3
:100A700005C02F3F19F00196A11DB11D3FBFBA2F30
:100A8000A92F982F8827BC01CD01620F711D811DF0
:100A9000911D42E0660F771F881F991F4A95D1F775
:100AA00008958F929F92AF92BF92CF92DF92EF9272
:100AB000FF926B017C010E942C054B015C01C1146B
:100AC000D104E104F104B9F00E942C0568197909F8
:100AD0008A099B09683E73408105910580F321E0F6
:100AE000C21AD108E108F10888EE880E83E0981E4A
:100AF000A11CB11CE4CFFF90EF90DF90CF90BF908E
:100B0000AF909F908F900895089520917F01260FB8
:100B10003327331F21323105ECF42091E002FC0130
:100B200090E080E0243069F082E00895A0917F0198
:100B30002191AC01415A5E4FA40FB52FB11D2C93EA
:100B40000196861798F380917F01680F60937F016B
:100B500080E0089581E008951092E00281E08093A2
:100B6000DF021092BA0261E082E10E94300261E08D
:100B700083E10E943002E9EBF0E080818E7F808388
:100B800080818D7F808388E48093B80085E48093A2
:100B9000BC000895CF93DF9391E090935E0188238A
:100BA000B9F0C091B800D091BA008091BC008A7BA6
:100BB0008093BC0060E082E10E94300260E083E14B
:100BC0000E9430020E94AC05D093BA00C093B800D6
:100BD000DF91CF910895CF92DF92EF92FF920F9322
:100BE0001F93CF93DF93D091090381E0D13208F0B6
:100BF0009CC0C09108030E942C056B017C01809170
:100C0000E00281116CC082E08093E00281E0809379
:100C1000DF028FEF8093DE021092DD02D093DC02C0
:100C2000A8EEB2E0ECEBF2E080E0D8138DC01092B9
:100C3000BB028091BB02CC0FC82BC093BB0280913A
:100C4000BA02813009F084C01092BA020E942C05C9
:100C50006B017C018091BB028093BB008091E2021A
:100C60009091E302A091E402B091E502892B8A2BD6
:100C70008B2BA1F00E942C050091E2021091E3025F
:100C80002091E4023091E5026C197D098E099F09DB
:100C9000061717072807390708F442C08091BC00DF
:100CA00083FDD8CF85EC8093BC000E942C056B019E
:100CB0007C018091E002823009F44CC08091DE0218
:100CC0008F3F09F469C08091DE02803209F466C06A
:100CD0008091DE02803309F463C084E026C08091F5
:100CE000E2029091E302A091E402B091E502892B27
:100CF0008A2B8B2B09F483CF0E942C050091E202F2
:100D00001091E3022091E4023091E5026C197D0913
:100D10008E099F09061717072807390708F06FCFB4
:100D20008091E1020E94CA0585E01092E7021092CC
:100D300009031092E602DF91CF911F910F91FF906E
:100D4000EF90DF90CF9008959D9191938F5F6DCF3D
:100D500085EEA9CF8091E2029091E302A091E40296
:100D6000B091E502892B8A2B8B2B09F4A2CF0E942C
:100D70002C050091E2021091E3022091E4023091EF
:100D8000E5026C197D098E099F09061717072807C8
:100D9000390708F08ECFC4CF80E0C7CF82E0C5CF3F
:100DA00083E0C3CFCF92DF92EF92FF920F931F9316
:100DB000CF93DF93D82FC62F613208F098C00E94DE
:100DC0002C056B017C018091E00281116BC081E0F8
:100DD0008093E0028093DF029FEF9093DE021092F7
:100DE000DD029C0F9093DC028093BB028091BB02DA
:100DF000DD0FD82BD093BB028091BA02813009F06D
:100E000078C01092BA020E942C056B017C0180917F
:100E1000BB028093BB008091E2029091E302A0911B
:100E2000E402B091E502892B8A2B8B2BA1F00E9462
:100E30002C050091E2021091E3022091E40230912E
:100E4000E5026C197D098E099F0906171707280707
:100E5000390708F448C08091BC0083FDD8CF85ECE9
:100E60008093BC000E942C056B017C018091E00204
:100E7000813009F440C08091DD028C1710F4C091DC
:100E8000DD02ECEBF2E0AAE9B2E080E08C1355C0A1
:100E90008C2FDF91CF911F910F91FF90EF90DF90FA
:100EA000CF9008958091E2029091E302A091E40234
:100EB000B091E502892B8A2B8B2B09F484CF0E94F9
:100EC0002C050091E2021091E3022091E40230919E
:100ED000E5026C197D098E099F0906171707280777
:100EE000390708F070CF8091E1020E94CA05C0E086
:100EF000CFCF85EEB5CF8091E2029091E302A09131
:100F0000E402B091E502892B8A2B8B2B09F4AECF3A
:100F10000E942C050091E2021091E3022091E4026C
:100F20003091E5026C197D098E099F090617170794
:100F30002807390708F09ACFD6CF91919D938F5FFC
:100F4000A5CF0895E091990280919802E81730F4B6
:100F5000F0E0E656FD4F808190E008958FEF9FEF1F
:100F6000089590919902809198022FEF3FEF981782
:100F700048F4E92FF0E0E656FD4F208130E09F5F16
:100F800090939902C9010895CF92DF92EF92FF9258
:100F90000F931F93CF93DF937C01CB018A012091A4
:100FA000E602222389F0EB016B01C40ED51ECC159D
:100FB000DD0569F06991D701ED91FC910190F08117
:100FC000E02DC7010995F3CF642F0E948505C80164
:100FD000DF91CF911F910F91FF90EF90DF90CF9015
:100FE000089521E02093E60227E72093080310925A
:100FF000E7021092090342E050E0BC0187EA93E067
:101000000E94C4070E94EB05982F80933A0481E068
:10101000911180E00895CF93DF931F92CDB7DEB793
:1010200069832091E6022223F9F0209109032032FE
:1010300058F021E030E0FC013383228390E080E02F
:101040000F90DF91CF9108958091E702E82FF0E0B3
:10105000E851FD4F998190838F5F8093E7028093E1
:10106000090381E090E0ECCF61E0CE0101960E949F
:101070008505F7CFCF93C82F81E08093E60283E503
:10108000809308031092E702109209036DE287EA49
:1010900093E00E940B086C2F87EA93E00E940B08F4
:1010A000CF910C94EB0590E080E008958DEF90E0F7
:1010B0000E94E2018EEF90E00C94E2010F931F93E7
:1010C000CF93DF93D0E0C0E0FE01E65CFE4F849159
:1010D000FE01E459FE4F0491FE01E85AFE4F1491BF
:1010E000112309F44BC081110E940702E12FF0E0A7
:1010F000EE0FFF1FE25BFE4FA591B491EC91E02350
:1011000081E090E009F480E00E94E2012196CC3079
:10111000D105D1F68EEF90E00E94E201C0E08C2F65
:10112000806480937C0080917A00806480937A0050
:1011300080917A0086FDFCCF8091780060917900E3
:10114000762F682F072E000C880B990B0E943F1BEF
:1011500024E13EEA43EA50E40E94661D0E94D81D45
:10116000CB010E94E201CF5FC830C9F68EEF90E05C
:10117000DF91CF911F910F910C94E20180E090E0FC
:10118000C3CFEF92FF920F931F93CF93DF938C0106
:10119000F62E81E08093E60287E7809308031092A1
:1011A000E70210920903F801608187EA93E00E9448
:1011B0000B080E94EB0580933A04811124C0CF2DC7
:1011C0000F2C000CDD0B6F2D87E70E94D2061092CA
:1011D00099028093980290E0C817D907E9F7E02EAA
:1011E000C02FD12F87EA93E00E94B10789938C2FFB
:1011F0008E198F15BCF381E0DF91CF911F910F9174
:10120000FF90EF90089580E0F7CF0F931F93CF9357
:10121000DF9300D0CDB7DEB78B01898362E0CE01CA
:1012200001960E94C108882381F089819A819827BC
:1012300089279827F8019183808381E00F900F9090
:10124000DF91CF911F910F910895F80111821082C3
:10125000F5CF0F931F93CF93DF9300D0CDB7DEB7B9
:101260008B01898362E0CE0101960E94C108882328
:1012700081F089819A81982789279827F80191839D
:10128000808381E00F900F90DF91CF911F910F919C
:101290000895F80111821082F5CFCF93DF93EC010E
:1012A00060E08E810E94300261E08E810E943002F7
:1012B00060E08E810E9430028BE891E00197F1F7A7
:1012C000DF91CF910895CF92DF92EF92FF920F932B
:1012D0001F93CF93DF936C017C0187E0E80EF11C34
:1012E000D0E0C0E0062F10E0B8010C2E02C07595CA
:1012F00067950A94E2F76170F70181917F010E947E
:1013000030022196C430D10579F7C601DF91CF9123
:101310001F910F91FF90EF90DF90CF900C944D09AB
:10132000CF92DF92EF92FF920F931F93CF93DF93B1
:10133000EC01F62E642F8C810E9430028D818F3F4C
:1013400019F060E00E9430020F2D10E08F8584FFBD
:1013500025C06E0187E0C80ED11CF12CE12CB8012C
:101360000E2C02C0759567950A94E2F76170F6013C
:1013700081916F010E943002FFEFEF1AFF0A88E0AF
:10138000E816F10461F7CE01DF91CF911F910F9123
:10139000FF90EF90DF90CF900C944D09B80184E05E
:1013A000759567958A95E1F7CE010E9463096F2DC7
:1013B000CE01DF91CF911F910F91FF90EF90DF90C1
:1013C000CF900C94630940E0682F88ED93E00C9473
:1013D0009009CF93DF93623028F09091E7039860F3
:1013E0009093E7036093EB031092EC0390E49093E7
:1013F000ED038093EE03805C8093EF0361E08091C6
:10140000DC030E948A028091DD038F3F19F061E0C6
:101410000E948A0261E08091DE030E948A02C8ED88
:10142000D3E09E01285D33408091E70384FD0BC02B
:1014300084E090E021962817390744F461E08E811A
:101440000E948A02EECF88E090E0F4CF8BE39DE02B
:101450000197F1F760E08091DC030E94300260E0C8
:101460008091DE030E9430028091DD038F3F19F0EE
:1014700060E00E9430028091E70384FD39C063E0A0
:1014800088ED93E00E946309CBE4D6E4CE01019796
:10149000F1F763E088ED93E00E9463092197F1F78B
:1014A00063E088ED93E00E94630983E592E0019791
:1014B000F1F762E088ED93E00E9463098091E70311
:1014C00080620E94E30984E08093E8038CE00E943C
:1014D000E30981E00E94E3098BE39FE10197F1F7C3
:1014E00082E08093E90386E0DF91CF910C94E309D9
:1014F00080620E94E3098BE496E40197F1F7809102
:10150000E70380620E94E30983E592E00197F1F727
:101510008091E70380620E94E309D0CF41E00E94FE
:10152000900981E090E00895FB0101900020E9F727
:101530003197AF01461B570BDC01ED91FC91028006
:10154000F381E02D09948F929F92AF92BF920F93F7
:101550001F93CF93DF93CDB7DEB7A1970FB6F89463
:10156000DEBF0FBECDBF19A2423008F44AE08E01A3
:101570000F5D1F4F842E912CB12CA12CA50194013D
:101580000E94C81CE62FB901CA01EA3004F5E05DEB
:10159000D801EE938D01232B242B252B79F790E096
:1015A00080E0109729F0BD018AE093E00E94940A40
:1015B000A1960FB6F894DEBF0FBECDBFDF91CF91DD
:1015C0001F910F91BF90AF909F908F900895E95C0D
:1015D000DFCFCF92DF92EF92FF92CF93DF936B0139
:1015E0007C016DE28AE093E00E949501EC016627A0
:1015F0007727CB016C197D098E099F094AE00E946B
:10160000A30A8C0F9D1FDF91CF91FF90EF90DF9089
:10161000CF900895BC01990F880B990B97FD0C94FE
:10162000E90A4AE00C94A30A4F925F926F927F926C
:101630008F929F92AF92BF92CF92DF92EF92FF92E2
:101640000F931F93CF936B017C01742EAC019B0110
:101650000E94631E6FE371E0811126C046015701AD
:10166000E894B7F82FEF3FEF4FE75FE7C501B4010C
:101670000E94631E81110CC02FEF3FEF4FE75FE721
:10168000C501B4010E94381B63E471E0181664F0D0
:101690002FEF3FEF4FE75FE4C701B6010E940E1E38
:1016A0001816ACF467E471E08AE093E0CF911F91E3
:1016B0000F91FF90EF90DF90CF90BF90AF909F90F1
:1016C0008F907F906F905F904F900C94940A2FEFC3
:1016D0003FEF4FE75FECC701B6010E94381B87FD63
:1016E000E1CF20E030E0A901C701B6010E94381B1C
:1016F00010E000E087FF0AC06DE28AE093E00E94FC
:1017000095018C01F7FAF094F7F8F094C0E060E0EE
:1017100070E080E09FE37C1641F020E030E040E2A2
:1017200051E40E94661DCF5FF6CFA70196010E948B
:10173000FA1C2B013C010E94DF1D4B015C014AE0B9
:101740000E94A30A7C01E00EF11ECC23C1F1C50169
:10175000B4010E943D1B9B01AC01C301B2010E9478
:10176000F91C4B015C016EE28AE093E00E94950156
:10177000E80EF91EC15018F120E030E040E251E4DB
:10178000C501B4010E949E1B2B013C010E94DF1D7C
:101790004B01B12CA12C4AE0C501B4010E94A30A5F
:1017A000E80EF91EC501B4010E943D1B9B01AC016E
:1017B000C301B2010E94F91C4B015C01DBCFC701E0
:1017C000CF911F910F91FF90EF90DF90CF90BF903E
:1017D000AF909F908F907F906F905F904F90089503
:1017E00085ED8093BC008091E2029091E302A0918C
:1017F000E402B091E5020796A11DB11D23E0B69564
:10180000A795979587952A95D1F72091BC0024FD3F
:1018100003C01092E00208954091E2025091E30269
:101820006091E4027091E502452B462B472B69F34A
:101830000097A105B10541F025E32A95F1F70000D5
:101840000197A109B109E1CF8091E1020C94CA0589
:10185000EF92FF920F931F93CF93DF937C01C09180
:10186000BC019091BD0102ED11E030E020E070E09C
:1018700060E042E050E080E0F801A191B1918F0179
:10188000AF3FB10541F1AE3FB10529F46F5F7F4F26
:101890004F5F5F4FF1CF6E157F05D1F7811102C009
:1018A000C42F952FE0915F04F09160042E173F073D
:1018B00030F4E0915B04F0915C04309749F41092AD
:1018C0005C01ECE5F1E0A0832F5F3F4F81E0E0CFCA
:1018D000E20FF31FF8CFC093BC019093BD0180913C
:1018E0005F04909160042817390740F480915B04ED
:1018F00090915C04280F391F892B21F410925C0110
:101900002CE531E0F9011082C0915B04D0915C04B8
:1019100060E070E0CB01209719F0CE010E948B1996
:101920007093BF016093BE0160E070E0CB0120972F
:1019300019F0CE010E9487196093C0017093C10114
:101940008093C2019093C301DF91CF911F910F91BA
:10195000FF90EF9008951F920F920FB60F921124EF
:101960002F933F934F935F936F937F938F939F93A7
:10197000AF93BF93EF93FF938091B4019091B50122
:10198000A091B601B091B701892B8A2B8B2BD1F195
:101990009091B301E091B101F091B201808189276A
:1019A00080838091B4019091B501A091B601B0916E
:1019B000B701181619061A061B069CF48091B4018B
:1019C0009091B501A091B601B091B7010197A1091D
:1019D000B1098093B4019093B501A093B601B0937F
:1019E000B701FF91EF91BF91AF919F918F917F913F
:1019F0006F915F914F913F912F910F900FBE0F907C
:101A00001F901895809100010E945E02EACF1F92FC
:101A10000F920FB60F9211242F933F934F935F9322
:101A20006F937F938F939F93AF93BF93EF93FF93A6
:101A30008AE093E00E947301FF91EF91BF91AF9113
:101A40009F918F917F916F915F914F913F912F91D6
:101A50000F900FBE0F901F9018951F920F920FB608
:101A60000F9211242F938F939F93EF93FF93E09105
:101A70001A03F0911B038081E0912003F091210370
:101A800082FD1BC09081809123038F5F8F73209113
:101A90002403821741F0E0912303F0E0E65FFC4F5E
:101AA000958F80932303FF91EF919F918F912F91B9
:101AB0000F900FBE0F901F9018958081F4CF1F924A
:101AC0000F920FB60F9211242F933F938F939F93F2
:101AD000AF93BF938091B8019091B901A091BA01E1
:101AE000B091BB013091A20123E0230F2D3758F5AF
:101AF0000196A11DB11D2093A2018093B80190937E
:101B0000B901A093BA01B093BB018091A301909158
:101B1000A401A091A501B091A6010196A11DB11D3E
:101B20008093A3019093A401A093A501B093A60173
:101B3000BF91AF919F918F913F912F910F900FBEC9
:101B40000F901F90189526E8230F0296A11DB11D36
:101B5000D2CF1F920F920FB60F9211242F933F9363
:101B60004F935F936F937F938F939F93AF93BF93A5
:101B7000EF93FF938091B900887F803609F44AC0C3
:101B8000F0F5883209F4A7C018F5803109F49BC03C
:101B9000B8F4882309F4F9C0883009F494C0FF919F
:101BA000EF91BF91AF919F918F917F916F915F91D5
:101BB0004F913F912F910F900FBE0F901F9018954E
:101BC000883109F488C0803251F78093DE0214C056
:101BD000803409F49DC040F48033B9F38833F9F6BA
:101BE0008093DE0285ECB0C0803509F485C088356D
:101BF00009F496C0883499F60E94F00BD0CF88394A
:101C000009F48CC038F5883729F050F4883611F083
:101C1000803729F683E08093E0021092A10157C03B
:101C2000883809F47BC0803919F0803809F0B7CFC3
:101C30008091A101803208F071C0E091A10181E0A2
:101C40008E0F8093A1018091BB00F0E0EF57FE4F13
:101C500080833DC0803B39F0E0F4803A09F479C0DC
:101C6000883A09F09CCF84E08093E00210928001D2
:101C700010927F01E091C601F091C7010995809112
:101C80007F0181110FC081E080937F0110925F017D
:101C900009C0803C09F4A6CF883C09F4A3CF883B57
:101CA00009F07DCFE091800181E08E0F809380016B
:101CB000F0E0E15AFE4F80818093BB00909180015B
:101CC00080917F0129C08091BB028093BB0085EC8D
:101CD0008093BC0064CF9091DD028091DC02981764
:101CE00058F5E091DD0281E08E0F8093DD02F0E097
:101CF000E454FD4F8081E9CFE091DD0281E08E0F59
:101D00008093DD028091BB00F0E0E454FD4F8083BE
:101D10009091DD028091DC029817C8F285E8D8CF57
:101D2000E091DD0281E08E0F8093DD028091BB00A7
:101D3000F0E0E454FD4F80838091DF0281115CCF9D
:101D400081E08093BA0284EA8093BC001092E002A2
:101D500026CF85EC8093BC001092E0028091A10117
:101D6000803230F4E091A101F0E0EF57FE4F108295
:101D70006091A10170E0E091C401F091C50181E89A
:101D800091E009951092A1010ACF1092DE0234CFA2
:101D90001F920F920FB60F9211242F933F934F93E0
:101DA0005F936F937F938F939F93AF93BF93CF93E3
:101DB000DF93EF93FF9380915D01C091D703D0E053
:101DC00087FF24C0109285001092840080915D01ED
:101DD0008F5F80935D0180915D01082E000C990B4F
:101DE0008C179D0724F480915D018C30C4F18091A3
:101DF000840090918500049680349C4908F47AC050
:101E00008091840090918500049676C080915D0158
:101E1000082E000C990B8C179D07C4F6E0915D010C
:101E20008E2FEE0F990BFC01EE0FFF1FE80FF91F2D
:101E3000ED54FC4F808186FFC9CFE0915D018E2F6C
:101E4000EE0F990BFC01EE0FFF1FE80FF91FED5489
:101E5000FC4F808160E08F730E943002B7CF2091E9
:101E6000840030918500E0915D018E2FEE0F990B7B
:101E7000FC01EE0FFF1FE80FF91FED54FC4F8181AD
:101E80009281820F931F9093890080938800E09144
:101E90005D018E2FEE0F990BFC01EE0FFF1FE80F77
:101EA000F91FED54FC4F808186FF11C0E0915D0168
:101EB0008E2FEE0F990BFC01EE0FFF1FE80FF91F9D
:101EC000ED54FC4F808161E08F730E943002FF91DE
:101ED000EF91DF91CF91BF91AF919F918F917F91C2
:101EE0006F915F914F913F912F910F900FBE0F9087
:101EF0001F90189580E49CE9909389008093880056
:101F00008FEF80935D01E3CFCF92DF92EF92FF924C
:101F10000F931F93E82FF92F05C0015011092109D4
:101F2000310961F1908196239417B9F305C00150EE
:101F300011092109310911F1908196239413F7CFEA
:101F4000C12CD12CE12CF12C0AC08FEFC81AD80A71
:101F5000E80AF80A0C151D052E053F0579F0808169
:101F60008623841791F36C2D7D2D8E2D9F2D1F912F
:101F70000F91FF90EF90DF90CF90089560E070E0B8
:101F800080E090E01F910F91FF90EF90DF90CF9055
:101F9000089510920D0310920C0388EE93E0A0E0D8
:101FA000B0E080930E0390930F03A0931003B093BF
:101FB000110323E131E030930B0320930A0325EC56
:101FC00030E0309317032093160324EC30E0309375
:101FD00019032093180320EC30E030931B03209367
:101FE0001A0321EC30E030931D0320931C0322ECF4
:101FF00030E030931F0320931E0326EC30E0309333
:1020000021032093200310922303109224031092A3
:102010002503109226031092AA031092A90380931D
:10202000AB039093AC03A093AD03B093AE0385E2F2
:1020300091E09093A8038093A70310925C04109200
:102040005B0410925E0410925D0410926004109282
:102050005F0461E170E090E080E00E94D42000978E
:1020600019F190935C0480935B0420E130E030939D
:102070005E0420935D0420915F0430916004232B63
:1020800011F4FC01108280E190E090936004809351
:102090005F046BE471E080915B0490915C040E94AA
:1020A0009A2116C020832EC080915B0490915C041D
:1020B000009711F00E944B2010925C0410925B0478
:1020C0001092600410925F0410925E0410925D04FE
:1020D000EFE4F4E02FEF48EB5BE08091D7038C3026
:1020E00008F791E0980F9093D703808390E0DC018C
:1020F000AA0FBB1FA80FB91FAD54BC4F12965C931B
:102100004E931197339684E0EB35F80731F781E071
:1021100080933B0410923C0483EC9BEAA6E7BBE36C
:1021200080933D0490933E04A0933F04B0934004F9
:1021300088ED9BE6A6E7BBE38093410490934204BD
:10214000A0934304B093440482EF94EEA4E6BBE36F
:102150008093450490934604A0934704B0934804A9
:102160001092DB031092DA0387E391E09093D90396
:102170008093D80387E08093DC038FEF8093DD03A7
:1021800088E08093DE0389E08093DF038AE0809318
:10219000E0038BE08093E1038CE08093E2031092F4
:1021A000E3031092E4031092E5031092E603109209
:1021B000E70361E080E10C94E909CF93DF93CDB7A9
:1021C000DEB72B970FB6F894DEBF0FBECDBF789465
:1021D00084B5826084BD84B5816084BD85B582602C
:1021E00085BD85B5816085BD80916E0081608093DD
:1021F0006E00109281008091810082608093810046
:102200008091810081608093810080918000816055
:10221000809380008091B10084608093B1008091B0
:10222000B00081608093B00080917A0084608093D8
:102230007A0080917A00826080937A0080917A009F
:10224000816080937A0080917A00806880937A0020
:102250001092C100E0911A03F0911B0382E0808389
:10226000E0911603F09117031082E0911803F091AA
:102270001903108210922203E0911E03F0911F03B4
:1022800086E08083E0911C03F0911D0380818061D2
:102290008083E0911C03F0911D038081886080831E
:1022A000E0911C03F0911D03808180688083E091A0
:1022B0001C03F0911D0380818F7D808368E8262EAA
:1022C000312C8AE093E00E945301892BD1F31092C4
:1022D00097021092960210E000E08AE093E00E94DC
:1022E0005301181619062CF10F3F110511F5009135
:1022F000CE011091CF01E090D001F090D101C80142
:102300000E94E201C7010E94E201093C110571F53A
:10231000EF28A9F50E945E0883E090E00E94E201A8
:1023200081E090E00E94E20186E190E00E94E201FB
:1023300026C08AE093E00E945301181619066CF635
:102340008AE093E00E9431018C0180919602909185
:102350009702FC01EE0FFF1FE253FE4F1183008333
:1023600001969093970280939602B7CF0A3C11058D
:1023700009F061C1E114F104B9F40E945E088EEF26
:1023800090E00E94E2018FEF90E00E94E20180E085
:1023900090E0892B09F495CF0E945F01882309F40E
:1023A0008DCF0E9400008ACF21E0E216F10411F5E2
:1023B00042EDE42E41E0F42E10E000E0D7018D91D3
:1023C0009D917D018F3F9105C1F28E3F910519F4DA
:1023D0000F5F1F4FF3CF61E00115110541F060E081
:1023E0000130110521F00230110541F762E00E9431
:1023F0008A02E4CFB2E0EB16F104F9F432EDE32EF9
:1024000031E0F32E10E000E0F701819191917F011E
:102410008F3F910509F4B1CF8E3F910519F40F5FFD
:102420001F4FF2CF60E00115110521F001301105B9
:1024300059F761E00E943002E7CFF3E0EF16F104B4
:1024400009F077C00EEC11E0D8011496ED90FC90E5
:10245000BFEFEB16F10409F492CFF80166817781A2
:10246000072E000C880B990B0E943F1B29EC38ECBF
:1024700048E45FE30E94661D0E94D81D4B016B017A
:1024800061E08E2D0E948A028114910429F460E09B
:102490008E2D0E9430022BC0FFEF8F16910411F495
:1024A00061E0F6CFF701FF27E65CFE4FE491E330F1
:1024B00031F148F4E130B9F0E230E1F020E8C21641
:1024C000D10474F7E4CFE73021F1E83051F1E43082
:1024D000A9F78091800080628093800090928B00A9
:1024E00080928A0004C084B5806884BD87BC0A5F7E
:1024F0001F4FAACF84B5806284BD88BCF8CF80917D
:10250000800080688093800090928900809288008B
:10251000EECF8091B00080688093B0008092B300CD
:10252000E6CF8091B00080628093B0008092B400CA
:10253000DECF34E0E316F10479F490E080E00E940D
:10254000280C6091BE017091BF01072E000C880B12
:10255000990B0E94510511CF45E0E416F104A1F456
:1025600090E080E00E94280C8091BE019091BF0114
:102570008230910508F401CF880F991F880F991FA9
:1025800005970197F1F7F9CE56E0E516F10489F4C5
:102590000E945E082FB7F8946091B8017091B9015C
:1025A0008091BA019091BB012FBF4AE00E94A30A1B
:1025B000E6CE87E0E816F10429F40E945E080E9446
:1025C0002C05F3CF98E0E916F10459F5F090D2010B
:1025D00081E090E00E94280C0091BE011091BF01A3
:1025E00082E090E00E94280CE091BC01F091BD01D6
:1025F000EE0FFF1FE253FE4F8081918120E030E01B
:10260000A9018D3F910541F02091BE013091BF019C
:10261000032E000C440B550BB8018F2D0E94C602EF
:10262000ACCEA9E0EA16F10409F0A9CE8091D2015E
:102630000E945E02A2CE043D110509F082C3E1149E
:10264000F10409F045C01091D20160E0812F0E9491
:10265000300283E090E00197F1F761E0812F0E9462
:10266000300283E290E00197F1F760E0812F0E9451
:1026700030028091D4019091D5019927FC01E45951
:10268000FE4F6491FC01E85AFE4FE491F0E0EE0F3A
:10269000FF1FE25BFE4F8591949100E412E42FE06E
:1026A00030E0462F0E94840F6B017C01C114D104DD
:1026B000E104F10439F0BFEFCB1ADB0AEB0AFB0AA5
:1026C000EFE0FE220E945E084AE0C701B6016ECF2D
:1026D000FAE0EF16F10409F090C1109299021092FD
:1026E00098021092E702109209030E94AC0523EFB2
:1026F00030E03093C7012093C60144EF50E050937F
:10270000C5014093C40160EF73E08AEA0E94290981
:10271000882309F46FC162EF73E08CEA0E942909F3
:10272000882309F467C164EF73E08EEA0E942909E7
:10273000882309F45FC160E074E080EB0E94050922
:10274000882309F457C162E074E082EB0E94050916
:10275000882309F44FC164E074E084EB0E9405090A
:10276000882309F447C166EF73E086EB0E942909CC
:10277000882309F43FC168EF73E088EB0E942909C0
:10278000882309F437C16AEF73E08AEB0E942909B4
:10279000882309F42FC16CEF73E08CEB0E942909A8
:1027A000882309F427C16EEF73E08EEB0E9429099C
:1027B000882309F41FC16091F4037091F503072E7B
:1027C000000C880B990B0E943F1B20E030E040EA90
:1027D0005BE30E949E1B2B013C0160910004709101
:1027E000010490E080E00E943D1B2FE632E143E0CF
:1027F00053E30E949E1B6B017C016091F603709174
:10280000F703072E000C880B990B0E943F1B20E05A
:1028100030E048EC57E30E949E1B4B015C01609145
:1028200002047091030490E080E00E943D1B2DECB7
:102830003CEC4CE454E30E949E1B609306047093AE
:102840000704809308049093090460910404709134
:10285000050490E080E00E943D1B60930A047093A1
:102860000B0480930C0490930D046091FC03709111
:10287000FD03072E000C880B990B0E943F1B2AE0DA
:1028800037ED43EA5DE30E949E1B60930E04709354
:102890000F0480931004909311046091FE037091D3
:1028A000FF03072E000C880B990B0E943F1B20E0B2
:1028B00030E040E253E40E94661D6093120470937E
:1028C000130480931404909315046091F0037091A5
:1028D000F103072E000C880B990B0E943F1B60939D
:1028E0001604709317048093180490931904609150
:1028F000F2037091F303072E000C880B990B0E94D2
:102900003F1B20E030E040EA5CE30E949E1B6093A6
:102910001A0470931B0480931C0490931D0460910F
:10292000F8037091F903072E000C880B990B0E9495
:102930003F1B20E030E048E45AE30E949E1B609376
:102940001E0470931F04809320049093210420E0C0
:1029500030E040E057E4C701B6010E949E1B60933F
:102960002204709323048093240490932504A701E8
:102970009601C301B2010E949E1B609326047093CE
:1029800027048093280490932904A5019401C7018A
:10299000B6010E949E1B60932A0470932B048093BF
:1029A0002C0490932D048CEE91E5A7E1B0E4809384
:1029B0002E0490932F04A0933004B093310420E3AD
:1029C00034E34EE75FE320933204309333044093C3
:1029D00034045093350480E097E5A4E9B6E380938E
:1029E000360490933704A0933804B093390481E0FF
:1029F00090E09CCC90E080E099CC9BE0E916F1045B
:102A000009F0BDCC0E945E0890E080E00E94280C96
:102A10002091C0013091C1014091C2015091C30188
:102A20002C833D834E835F8384EF89838EE28A8388
:102A3000CE0101960E94F107811103C00E94560841
:102A40007AC065E070E080E090E00E94510586EF7A
:102A5000898362E0CE0101960E94C108882371F348
:102A6000698170E090E080E00E943F1B20E030E050
:102A700040E853E40E949E1B6B017C016A8170E078
:102A800090E080E00E943F1B9B01AC01C701B601B2
:102A90000E94FA1C20910A0430910B0440910C040E
:102AA00050910D040E94F91C2091060430910704F6
:102AB00040910804509109040E949E1B6B017C0107
:102AC0002091120430911304409114045091150484
:102AD0000E94FA1C9B01AC0160910E0470910F04DE
:102AE00080911004909111040E94661DA701960127
:102AF0000E94FA1C6B017C0141E00E94140B8EEFD6
:102B000090E00E94E20184EF89838A83CE010196DE
:102B10000E94F107882379F06AE170E080E090E09C
:102B20000E94510586EF898363E0CE0101960E94E1
:102B3000C108811105C00E9456080E9456081FCC8A
:102B400020E030E048EC51E4C701B6010E94F91CD6
:102B50006B017C01AC019B010E949E1B2B013C017F
:102B6000698170E090E080E00E943F1B20E030E04F
:102B700040E853E40E949E1B4B015C016A8170E0B7
:102B800090E080E00E943F1B9B01AC01C501B401B5
:102B90000E94FA1C4B015C016B8170E090E080E0C8
:102BA0000E943F1B20E030E040E85BE30E949E1B58
:102BB0009B01AC01C501B4010E94FA1C4B015C01F0
:102BC00020911E0430911F04409120045091210453
:102BD000C301B2010E949E1B688779878A879B8701
:102BE00020911A0430911B0440911C0450911D0443
:102BF000C701B6010E949E1B9B01AC0168857985C7
:102C00008A859B850E94FA1C209116043091170436
:102C100040911804509119040E94FA1C9B01AC01C8
:102C2000C501B4010E94F91C4B015C0120912A04EA
:102C300030912B0440912C0450912D04C301B2011A
:102C40000E949E1B2B013C012091260430912704F9
:102C50004091280450912904C701B6010E949E1B8F
:102C60009B01AC01C301B2010E94FA1C2091220415
:102C70003091230440912404509125040E94FA1CB1
:102C80009B01AC01C501B4010E94661D6B017C0172
:102C9000AC019B010E949E1B2091360430913704A9
:102CA00040913804509139040E949E1B4B015C01F5
:102CB0002091320430913304409134045091350412
:102CC000C701B6010E949E1B9B01AC01C501B40166
:102CD0000E94FA1C20912E0430912F044091300460
:102CE000509131040E94FA1C6B017C0142E00E9469
:102CF000140B8EEF90E00E94E20120E03AE24DE2F8
:102D000057E46C817D818E819F810E94661D9B01AD
:102D1000AC0160E070E080E89FE30E94F91C26EFC0
:102D200038E248EA50E40E94131E9B01AC01C7013F
:102D3000B6010E94661D42E00E94140B8EEF90E0E7
:102D4000F5CA0E3D110509F01ACBE114F10409F0A2
:102D500080C0E1E0F1E0F12CE12C819191910196AC
:102D600009F073C06701CC0CDD1C86010E0D1F1D20
:102D7000015B1B4FD8018C918C3008F05CC0B09087
:102D8000D20161E08B2D0E948A02F8018081282FF8
:102D900030E0F901EE0FFF1FE20FF31FED54FC4F7F
:102DA0002B2D2F73B22E9081907CB92AB082D8013E
:102DB00011961C92119712961C922CE0622F0E9481
:102DC0009D1F829FB001112430E020E0AB01420F33
:102DD000531FFA01EE0FFF1FE40FF51FED54FC4FD8
:102DE000908196FD16C02F5F3F4F2C30310571F753
:102DF00081110FC01092800082E0809381001092B8
:102E0000850010928400B19A80916F008260809357
:102E10006F00F601EE0DFF1DE15BFB4FE0818E2F91
:102E200090E0FC01EE0FFF1FE80FF91FED54FC4F7F
:102E3000808180648083F601EF5FFE4F8091D20134
:102E40009091D3019183808398CABFEFEB1AFB0A5C
:102E500084CFE1E0EE16F10409F097C02091D20191
:102E60003091D301E1E0F1E00FEF1FEF90E080E05F
:102E7000419151912417350709F48C010196853051
:102E80009105B1F70F3F100709F477CAA091D4015B
:102E9000B091D5017801EE0CFF1CA03222E0B20700
:102EA000E4F5F701E00FF11FE15BFB4F8181410188
:102EB000881A910887FD9394880C991C880C991C9A
:102EC000092C000CAA08BB08828128E532E0281BE7
:102ED000310987FD3395220F331F220F331F032E35
:102EE000000C440B550B281939094A095B09A53B0D
:102EF000B10514F0A4EBB0E0B7FF02C0B0E0A0E071
:102F00000E94891C24EB30E040E050E00E945F1CEE
:102F1000820E931EA41EB51ED4010E0D1F1DF801B6
:102F2000E15BFB4F20812C3008F027CA8181A10191
:102F3000481B510987FD5395CA01880F991F880FB7
:102F4000991FA817B90784F08281E8E5F2E0E81B31
:102F5000F10987FDF395CF01880F991F880F991FFD
:102F6000A817B9070CF4CD010297880F991F4FB726
:102F7000F89430E0F901EE0FFF1FE20FF31FED545C
:102F8000FC4F928381834FBFF8C9F2E0EF16F10442
:102F900009F07BC02091D2013091D301A1E0B1E0D2
:102FA000EFEFFFEF90E080E04D915D912417350742
:102FB00009F4FC01019685309105B1F710E000E0BD
:102FC000EF3FFE0709F45AC0CF01880F991FE80FA1
:102FD000F91FE15BFB4F8281B8E5CB2EB2E0DB2E1F
:102FE000C81AD10887FDD394CC0CDD1CCC0CDD1C99
:102FF0000D2C000CEE08FF0881814101881A910810
:1030000087FD9394880C991C880C991C092C000C42
:10301000AA08BB0880818F3FA9F190E0FC01EE0F68
:10302000FF1FE80FF91FED54FC4F8181928173E07F
:10303000880F991F7A95E1F7B0E0A0E0E4E0B5953C
:10304000A79597958795EA95D1F702969C012F5FF2
:103050003F4F032E000C440B550B281939094A0920
:103060005B09A4EBB0E00E947E1CA7019601281921
:1030700039094A095B090E945F1C89010E945E08A8
:10308000C80154C990E080E0E1CF33E0E316F104D9
:10309000B1F54091D2015091D301E1E0F1E08FEF21
:1030A0009FEF30E020E0619171914617570709F4D6
:1030B000C9012F5F3F4F25303105A9F78F3F980792
:1030C00009F45BC99C01220F331F820F931FFC017F
:1030D000E15BFB4FE0818E2F90E0FC01EE0FFF1FC4
:1030E000E80FF91FED54FC4F80818F7B80832F5FA9
:1030F0003E4FEFEFFFEFD901ED93FC933EC9FAE0AD
:10310000EF16F10401F510929902109298021092B4
:10311000E702109209030E94AC0523EF30E03093E0
:10312000C7012093C60144EF50E05093C50140937E
:10313000C40180E00E943A0880E10E943A0888E0D9
:103140000E943A081AC95BE0E516F10409F071C063
:1031500011E01093E60283E5809308031092E702E2
:103160001092090362E387EA93E00E940B080E9431
:10317000EB051093E6021092E7021092090366E055
:1031800083E50E94D206F82E10929902809398024D
:103190000BE314E0C8018B5394400F5F1F4F209145
:1031A0009902F21641F087EA93E00E94B107D80134
:1031B0001D968C93EFCF069729F010923B0481E087
:1031C00080933C040E94EB058091490490914A044D
:1031D0009093CD018093CC0180914B0490914C044D
:1031E0009093CB018093CA0180914D0490914E043D
:1031F0009093C9018093C8010E945E088091CC0120
:103200009091CD010E940A0B8EEF90E00E94E201A6
:103210008091CA019091CB010E940A0B8EEF90E041
:103220000E94E2018091C8019091C9010E940A0B9D
:10323000A6C8B4E1EB16F10439F46091D401809191
:10324000D2010E94E9099BC8E5E1EE16F104B1F450
:103250008091D201E091D401E43008F0E3E0909154
:10326000EB03E91710F0EFEFE90FF0E0E852FC4F45
:103270009489890F80680E94E30981C8F6E1EF16FE
:10328000F10479F50DB71EB7A2EDB1E0FD0190E0B4
:1032900080E0219131912F3F310511F00196F9CF56
:1032A0002DB73EB7281B390B0FB6F8943EBF0FBEA3
:1032B0002DBF6DB77EB76F5F7F4FFB01860F971FE6
:1032C0008E179F0721F02C9112962193F9CF88ED4C
:1032D00093E00E94940A0FB6F8941EBF0FBE0DBF74
:1032E0004EC837E1E316F10409F049C881E00E94B5
:1032F000E3098BE39FE10197F1F741C880915B04FB
:1033000090915C04009711F00C944B20089566276F
:1033100077270C94C7191F93FC0199278827BC01B4
:10332000E89411911032E9F3193010F01E30C8F30F
:103330001B3251F01D3249F4689406C00E94B21944
:10334000610F711D811D911D119110531A30B0F341
:103350003EF490958095709561957F4F8F4F9F4F6C
:103360001F910895592F482F372F262F660F771F4B
:10337000881F991F660F771F881F991F620F731F81
:10338000841F951F660F771F881F991F0895B0E04F
:10339000A0E0EDECF9E10C94971C5C017B01611558
:1033A000710519F0DB018D939C9385010F5F1F4F11
:1033B000F501D0818D2F90E00E94171B6C01892BA5
:1033C000B9F5DD32B9F50F5F1F4FD5011196DC91CC
:1033D000C1E05801F1E0AF1AB10843E050E062EFFC
:1033E00070E0C5010E94201B892B69F5680182E00D
:1033F000C80ED11C45E050E06DEE70E0C6010E94A1
:10340000201B892B21F4680197E0C90ED11CE1141F
:10341000F10419F0D701CD92DC9260E070E080E811
:103420009FEFC111FFC060E070E080E89FE7FAC045
:103430005801BBCFDB3229F485010E5F1F4FF50128
:10344000D181C0E0C6CF43E050E06AEE70E0C50134
:103450000E94201B892BE9F0F80110E000E020E039
:1034600030E0A9015F01B0ED8B2E8D0E89E088154B
:10347000C8F19C2E689491F88C2F8870C2FF16C0FA
:10348000811102C00F5F1F4F3196D501DC91C92D0C
:10349000E9CFE114F10429F00E5F1F4FF70111830A
:1034A000008360E070E080EC9FE7BCC0882311F0EF
:1034B00001501109A5E0B0E00E947E1C9B01AC0107
:1034C000220F331F441F551F280D311D411D511D53
:1034D000283999E93907490799E15907A8F2C660DF
:1034E0009C2ED2CFAEEF8A1206C0C3FD3CC09C2EEC
:1034F000689493F8C9CFDF7DD534A9F580818D32EA
:1035000039F4C061DF011296818162E070E006C08B
:10351000DF018B32C1F3119661E070E080535D01F1
:10352000A61AB70A8A30F8F4E0E8CE16ECE0DE0618
:103530005CF4B601660F771F660F771FC60ED71EA5
:10354000CC0CDD1CC80ED11C5D01FFEFAF1ABF0A09
:103550008C9180538A30A8F1C4FF03C0D194C194E8
:10356000D1080C0D1D1DC1FF09C0E114F10431F09B
:1035700081E0A81AB108D701AD92BC92CA01B90185
:103580000E943D1BC370C33009F490584B015C018D
:1035900020E030E0A9010E94381B882309F440C0D4
:1035A000C1E2D1E017FF05C0119501951109C9E0ED
:1035B000D1E06E01B8E1CB1AD10880E2E82EF12CFF
:1035C0000FC0D501B1CFFE012591359145915491A0
:1035D0000E191F09C501B4010E949E1B4B015C011D
:1035E000D501C4010E151F0574F72497F594E794CF
:1035F000CC16DD06A9F78A2F880F8B2F881F8F3FE7
:1036000049F020E030E0A901C501B4010E94381B57
:10361000811106C082E290E090936204809361047D
:10362000C501B401CDB7DEB7ECE00C94B31C911129
:103630000C940B1C803219F089508550C8F70895FE
:10364000FB01DC014150504088F08D9181341CF029
:103650008B350CF4805E659161341CF06B350CF495
:10366000605E861B611171F3990B0895881BFCCF76
:103670000E947A1B08F481E00895E89409C097FB42
:103680003EF490958095709561957F4F8F4F9F4F39
:103690009923A9F0F92F96E9BB279395F69587957D
:1036A00077956795B795F111F8CFFAF4BB0F11F440
:1036B00060FF1BC06F5F7F4F8F4F9F4F16C08823E7
:1036C00011F096E911C0772321F09EE8872F762F1D
:1036D00005C0662371F096E8862F70E060E02AF05E
:1036E0009A95660F771F881FDAF7880F969587954A
:1036F00097F90895990F0008550FAA0BE0E8FEEF1F
:1037000016161706E807F907C0F012161306E407A5
:10371000F50798F0621B730B840B950B39F40A269E
:1037200061F0232B242B252B21F408950A2609F47C
:10373000A140A6958FEF811D811D08950E94B11BA8
:103740000C94251C0E94171C38F00E941E1C20F0AF
:10375000952311F00C940E1C0C94141C11240C9441
:10376000591C0E94361C70F3959FC1F3950F50E0D1
:10377000551F629FF001729FBB27F00DB11D639F23
:10378000AA27F00DB11DAA1F649F6627B00DA11DC9
:10379000661F829F2227B00DA11D621F739FB00D6F
:1037A000A11D621F839FA00D611D221F749F3327DF
:1037B000A00D611D231F849F600D211D822F762F78
:1037C0006A2F11249F5750409AF0F1F088234AF055
:1037D000EE0FFF1FBB1F661F771F881F91505040C1
:1037E000A9F79E3F510580F00C940E1C0C94591CB7
:1037F0005F3FE4F3983ED4F3869577956795B79548
:10380000F795E7959F5FC1F7FE2B880F911D969561
:10381000879597F9089599278827089597F99F67BD
:1038200080E870E060E008959FEF80EC0895002448
:103830000A941616170618060906089500240A9415
:1038400012161306140605060895092E0394000C9B
:1038500011F4882352F0BB0F40F4BF2B11F460FF2A
:1038600004C06F5F7F4F8F4F9F4F089557FD905853
:10387000440F551F59F05F3F71F04795880F97FB34
:10388000991F61F09F3F79F08795089512161306EE
:103890001406551FF2CF4695F1DF08C0161617061D
:1038A0001806991FF1CF8695710561050894089552
:1038B000E894BB2766277727CB0197F90895052E53
:1038C00097FB1EF400940E94761C57FD07D00E94BF
:1038D000C81C07FC03D04EF40C94761C5095409500
:1038E000309521953F4F4F4F5F4F089590958095AC
:1038F000709561957F4F8F4F9F4F08950E94EA1CEE
:10390000A59F900DB49F900DA49F800D911D112433
:103910000895B7FF0C947E1C0E947E1C821B930BA3
:1039200008952F923F924F925F926F927F928F9263
:103930009F92AF92BF92CF92DF92EF92FF920F933E
:103940001F93CF93DF93CDB7DEB7CA1BDB0B0FB648
:10395000F894DEBF0FBECDBF09942A883988488805
:103960005F846E847D848C849B84AA84B984C8849B
:10397000DF80EE80FD800C811B81AA81B981CE0F92
:10398000D11D0FB6F894DEBF0FBECDBFED01089577
:10399000A1E21A2EAA1BBB1BFD010DC0AA1FBB1F53
:1039A000EE1FFF1FA217B307E407F50720F0A21BC5
:1039B000B30BE40BF50B661F771F881F991F1A9432
:1039C00069F760957095809590959B01AC01BD015C
:1039D000CF010895A29FB001B39FC001A39F700DB6
:1039E000811D1124911DB29F700D811D1124911D07
:1039F00008955058BB27AA270E94111D0C94251C1E
:103A00000E94171C38F00E941E1C20F039F49F3FC2
:103A100019F426F40C94141C0EF4E095E7FB0C94B6
:103A20000E1CE92F0E94361C58F3BA176207730761
:103A30008407950720F079F4A6F50C94581C0EF431
:103A4000E0950B2EBA2FA02D0B01B90190010C01AE
:103A5000CA01A0011124FF27591B99F0593F50F4C6
:103A6000503E68F11A16F040A22F232F342F44271E
:103A7000585FF3CF469537952795A795F040539516
:103A8000C9F77EF41F16BA0B620B730B840BBAF0E6
:103A90009150A1F0FF0FBB1F661F771F881FC2F751
:103AA0000EC0BA0F621F731F841F48F48795779565
:103AB0006795B795F7959E3F08F0B0CF9395880F1F
:103AC00008F09927EE0F9795879508950E947A1D23
:103AD0000C94251C0E941E1C58F00E94171C40F0DC
:103AE00029F45F3F29F00C940E1C51110C94591CC1
:103AF0000C94141C0E94361C68F39923B1F35523CF
:103B000091F3951B550BBB27AA27621773078407F0
:103B100038F09F5F5F4F220F331F441FAA1FA9F386
:103B200035D00E2E3AF0E0E832D091505040E69574
:103B3000001CCAF72BD0FE2F29D0660F771F881FD5
:103B4000BB1F261737074807AB07B0E809F0BB0BC8
:103B5000802DBF01FF2793585F4F3AF09E3F5105DC
:103B600078F00C940E1C0C94591C5F3FE4F3983EC3
:103B7000D4F3869577956795B795F7959F5FC9F7C5
:103B8000880F911D9695879597F90895E1E0660F46
:103B9000771F881FBB1F621773078407BA0720F0BF
:103BA000621B730B840BBA0BEE1F88F7E095089528
:103BB0000E94DF1D6894B1110C94591C08950E9455
:103BC0003E1C88F09F5798F0B92F9927B751B0F055
:103BD000E1F0660F771F881F991F1AF0BA95C9F791
:103BE00014C0B13091F00E94581CB1E008950C94BB
:103BF000581C672F782F8827B85F39F0B93FCCF36E
:103C0000869577956795B395D9F73EF4909580950D
:103C1000709561957F4F8F4F9F4F08950E947A1B3B
:103C200008F48FEF0895FA01EE0FFF1F309621057B
:103C30003105A1F16115710561F48038BFE39B077F
:103C400049F168949038810561F08038BFEF9B0797
:103C500041F099234AF5FF3FE1053105210519F1AE
:103C6000E8940894E795D901AA2329F4AB2FBE2F35
:103C7000F85FD0F310C0FF5F70F4A695E0F7F73956
:103C800050F019F0FF3A38F49F779F930DD00F90C2
:103C900007FC9058089546F00C94141C60E070E006
:103CA00080E89FE308954FE79F775F934F933F939B
:103CB0002F930E94131F2F913F914F915F910E946C
:103CC0009E1B0C94701E0E947A1B880B990B089502
:103CD00029F416F00C940E1C0C94581C0C94141C13
:103CE0000E943E1CA8F39638A0F707F80F92E894BC
:103CF0002BE33AEA48EB5FE70E94B41B0F920F9266
:103D00000F924DB75EB70F920E945B1FE8E6F0E09E
:103D10000E94A21E4F915F91EF91FF91E595EE1FDA
:103D2000FF1F49F0FE57E0684427EE0F441FFA9545
:103D3000E1F74195550B0E94D51E0F9007FE0C949C
:103D4000C91E0895DF93CF931F930F93FF92EF92B5
:103D5000DF927B018C01689406C0DA2EEF010E948D
:103D6000B11BFE01E894A59125913591459155919E
:103D7000A6F3EF010E94111DFE019701A801DA943C
:103D800069F7DF90EF90FF900F911F91CF91DF9136
:103D900008959B01AC0160E070E080E89FE30C9423
:103DA000661D0C940E1C0C948F1F0E943E1CD8F3B1
:103DB0009923C9F3940F511DA3F39150504094F0EF
:103DC00059F0882332F0660F771F881F91505040BA
:103DD000C1F79E3F51052CF7880F911D9695879549
:103DE00097F908955F3FACF0983E9CF0BB2786950D
:103DF00077956795B79508F4B1609395C1F7BB0FB8
:103E000058F711F460FFE8CF6F5F7F4F8F4F9F4FE0
:103E1000E3CF0C94591C16F00C948F1F0C94141CB7
:103E200068940C940E1C0E943E1CA8F39923C1F3C5
:103E3000AEF3DF93CF931F930F93FF92C92FDD272C
:103E400088232AF02197660F771F881FDAF720E072
:103E500030E040E85FEB9FE3883920F0803E38F0A7
:103E600021968F770E94FA1CE0E9F0E004C00E94DE
:103E7000FA1CEDEBF0E00E94A21E8B01BE01EC01EA
